:100000000C946B000C945C1E0C94891E0C94930051
:100010000C9493000C9493000C9493000C94930014
:100020000C9493000C9493000C9493000C94930004
:100030000C9493000C9455130C9493000C9493001F
:100040000C94B61E0C9493000C940E1A0C945C1A2B
:100050000C9493000C9493000C9493000C949300D4
:100060000C9493000C94930020557365206F6E657B
:10007000206F66200000000000240027002A0000F6
:10008000000000250028002B0000000000230026AF
:10009000002900040404040404040402020202020D
:1000A000020303030303030102040810204080013C
:1000B00002040810200102040810200000000700BC
:1000C0000201000003040600000000000000000020
:1000D000BA13C81BB31311241FBECFEFD8E0DEBF85
:1000E000CDBF12E0A0E0B1E0E0E5FAE402C0059087
:1000F0000D92A435B107D9F715E0A4E5B2E001C02F
:100100001D92A435B107E1F710E0C4EDD0E004C0C2
:100110002297FE010E94E024C03DD107C9F70E944A
:100120001E1C0C941B250C9400000F931F93CF935F
:10013000DF93689F8001699F100D789F100D112437
:10014000C8010E94B100EC01009729F060E070E066
:10015000A8010E94ED02CE01DF91CF911F910F9176
:100160000895CF93DF93BC018230910510F462E0D3
:1001700070E0A0915205B0915305ED01E0E0F0E090
:1001800040E050E021C0888199818617970769F483
:100190008A819B81309719F09383828304C0909366
:1001A000530580935205FE0134C06817790738F46F
:1001B0004115510519F08417950708F4AC01FE01AB
:1001C0008A819B819C01E9012097E9F6411551053F
:1001D000A9F1CA01861B970B049708F4BA01E0E065
:1001E000F0E02AC08D919C91119784179507F9F43E
:1001F0006417750781F412968D919C91139730972F
:1002000019F09383828304C0909353058093520521
:10021000FD0132964CC0CA01861B970BFD01E80F09
:10022000F91F6193719302978D939C9340C0FD01D8
:10023000828193819C01D9011097A1F6809150058C
:1002400090915105892B41F48091100290911102F7
:1002500090935105809350054091120250911302E2
:100260004115510541F44DB75EB780910E02909152
:100270000F02481B590B2091500530915105CA01BE
:10028000821B930B8617970780F0AB014E5F5F4F81
:100290008417950750F0420F531F50935105409318
:1002A0005005F9016193719302C0E0E0F0E0CF01E5
:1002B000DF91CF910895CF93DF93009709F450C059
:1002C000EC0122971B821A82A0915205B09153052E
:1002D000109709F140E050E0AC17BD0708F1BB836F
:1002E000AA83FE0121913191E20FF31FAE17BF07E0
:1002F00079F48D919C911197280F391F2E5F3F4FF4
:100300003983288312968D919C9113979B838A83BE
:100310004115510571F4D0935305C093520520C087
:1003200012968D919C911397AD01009711F0DC010D
:10033000D3CFFA01D383C28321913191E20FF31F0E
:10034000CE17DF0769F488819981280F391F2E5F46
:100350003F4FFA01318320838A819B81938382837B
:10036000DF91CF910895A0E0B0E0E9EBF1E00C94CB
:10037000E6246C01009729F4CB010E94B1006C01C6
:10038000C1C08EEF882E8FEF982E8C0C9D1C86019D
:10039000060F171F0815190508F4B2C0F401A08153
:1003A000B181A617B707B8F0A530B10508F4AAC007
:1003B000CD0104978617970708F4A4C01297A61BCF
:1003C000B70BF801A193B193D4016D937C93CF0146
:1003D0000E945B0197C07B01EA1AFB0AEEEFFFEF78
:1003E000EE0EFF1E36016A0E7B1EC0915205D091A3
:1003F000530544245524AA24BB244AC0C615D70556
:10040000E1F5488159814E155F05B8F1CA0104979D
:100410008E159F05B0F41296A40FB51FF401B18399
:10042000A0832A813B814114510431F0D2011396FB
:100430003C932E93129766C0309353052093520538
:1004400061C08A819B81F80193838283425050402E
:100450004E195F09518340834114510431F0D20198
:1004600013961C930E93129704C010935305009398
:100470005205F4017183608345C088819981A81673
:10048000B90608F45C012E018A819B819C01E90177
:10049000209709F0B3CF80915005909151058615B2
:1004A0009705E9F4A616B706D0F420911202309110
:1004B00013022115310541F42DB73EB780910E028C
:1004C00090910F02281B390B02171307C8F41093E1
:1004D000510500935005D4016D937C9313C0CB015B
:1004E0000E94B100EC01009759F0F4014081518164
:1004F000B6010E94D202C6010E945B016E0102C0D9
:10050000CC24DD24C601CDB7DEB7E0E10C94022592
:10051000FC0188279927E89421912032E9F32930BA
:1005200010F02E30C8F32B3241F02D3239F468949C
:1005300004C00E949703820F911D219120532A30FD
:10054000C0F31EF4909581959F4F08951F93FC0171
:1005500099278827BC01E89411911032E9F31930EA
:1005600010F01E30C8F31B3251F01D3249F468946C
:1005700006C00E948203610F711D811D911D1191A2
:1005800010531A30B0F33EF49095809570956195B4
:100590007F4F8F4F9F4F1F91089544E552E00E9477
:1005A0002F030895FB01DC0102C001900D92415020
:1005B0005040D8F708956817790768F4FB01DC010B
:1005C000E40FF51FA40FB51F02C002900E92415018
:1005D0005040D8F708950C94D202DC0101C06D930D
:1005E00041505040E0F70895FC018191861721F0B9
:1005F0008823D9F7992708953197CF010895FB01F2
:10060000DC0101900D920020E1F70895FB01DC016F
:100610004150504048F001900D920020C9F701C0B0
:100620001D9241505040E0F70895FB015191552330
:10063000A9F0BF01DC014D9145174111E1F759F4D3
:10064000CD010190002049F04D9140154111C9F3B1
:10065000FB014111EFCF81E090E0019708950097F1
:1006600031F4DA018D919C91009709F40EC0DC0100
:10067000FB013D912191222319F03217C9F3FACFE2
:10068000332331F4DA011D921C92882799270895AB
:100690001197AF93BF93FB013D912191321771F4F4
:1006A000332321F488279927119702C01E921196AF
:1006B000FA01A193B0839F918F910895222369F746
:1006C000EACFFB019F01E8944230C4F04532B4F414
:1006D0004A3029F497FB1EF4909581959F4F642F23
:1006E00077270E949524805D8A330CF0895D819381
:1006F000CB010097A1F716F45DE251931082C90176
:100700000C94CC05592F482F372F262F660F771FB3
:10071000881F991F660F771F881F991F620F731F0D
:10072000841F951F660F771F881F991F08957AE011
:10073000979F902D879F802D910D11240895FB0187
:100740009F01423074F0453264F4642F77270E9491
:100750009524805D8A330CF0895D8193CB010097ED
:10076000A1F71082C9010C94CC05AEE0B0E0EBEB30
:10077000F3E00C94F2240D891E8986E08C831A83A1
:1007800009838FEF9FE79E838D839E01275E3F4FF6
:10079000CE0101966F89788DA9010E94D9032F811E
:1007A0003885020F131FF80110822E96E4E00C9496
:1007B0000E25ABE0B0E0EFEDF3E00C94E4243C0157
:1007C0002B015A01FC0117821682838181FD03C02F
:1007D0006FEF7FEFC6C19AE0892E1E010894211C9D
:1007E000311CF3012381F20123FD859123FF8191C7
:1007F0002F01882309F4B2C1853239F423FD859194
:1008000023FF81912F01853229F490E0B3010E94EA
:10081000DC05E7CF982FFF24EE249924FFE1FF1594
:10082000D0F09B3269F09C3228F4903259F0933228
:1008300091F40EC09D3249F0903369F441E024C038
:1008400052E0F52A84E0F82A28C098E0F92A25C069
:10085000E0E1FE2A22C0F7FC29C0892F80538A30AC
:1008600070F4F6FE05C0989C902C1124980E15C0CB
:10087000E89CE02C1124E80EF0E2FF2A0EC09E3224
:1008800029F4F6FC6BC140E4F42A07C09C3619F445
:1008900050E8F52A02C0983649F4F20123FD9591FB
:1008A00023FF91912F01992309F0B8CF892F855407
:1008B000833018F08052833038F444E050E0A40EC6
:1008C000B51E5FE359830FC0933631F0933779F04B
:1008D000933509F056C020C0F5018081898342E03C
:1008E00050E0A40EB51E610101E010E012C0F50158
:1008F000C080D180F6FC03C06FEF7FEF02C0692D8E
:1009000070E042E050E0A40EB51EC6010E94C10591
:100910008C015FE7F52214C0F501C080D180F6FCA0
:1009200003C06FEF7FEF02C0692D70E042E050E03E
:10093000A40EB51EC6010E94B6058C0150E8F52A2A
:10094000F3FE07C01AC080E290E0B3010E94DC050C
:10095000EA948E2D90E008171907A8F30EC0F6014F
:10096000F7FC8591F7FE81916F0190E0B3010E9441
:10097000DC05E110EA94015010400115110579F7EA
:10098000EAC0943611F0993669F5F7FE08C0F50112
:10099000208131814281538184E090E00AC0F501D9
:1009A000808191819C01442737FD4095542F82E03E
:1009B00090E0A80EB91E9FE6F92257FF09C0509596
:1009C0004095309521953F4F4F4F5F4FE0E8FE2A0D
:1009D000CA01B901A1012AE030E00E940806D82E20
:1009E000D21840C0953729F41F2D1F7E2AE030E031
:1009F0001DC01F2D197F9F3661F0903720F4983568
:100A000009F0ACC00FC0903739F0983709F0A6C094
:100A100004C028E030E00AC0106114FD146020E139
:100A200030E004C014FD166020E132E017FF08C07A
:100A3000F501608171818281938144E050E008C0BA
:100A4000F50180819181BC0180E090E042E050E0BE
:100A5000A40EB51EA1010E940806D82ED2188FE759
:100A6000F82EF122F6FE0BC05EEFF522D91438F411
:100A7000F4FE07C0F2FC05C08FEEF82202C01D2D67
:100A800001C0192DF4FE0DC0FE01ED0DF11D808198
:100A9000803319F499EEF92208C01F5FF2FE05C0F9
:100AA00003C08F2D867809F01F5F0F2DF3FC14C053
:100AB000F0FE0FC01E1510F09D2C0BC09D2C9E0C3F
:100AC000911A1E2D06C080E290E0B3010E94DC0561
:100AD0001F5F1E15C0F304C01E1510F4E11A01C0FB
:100AE000EE2404FF0FC080E390E0B3010E94DC0518
:100AF00002FF1DC001FD03C088E790E00EC088E53D
:100B000090E00BC0802F867891F001FF02C08BE24D
:100B100001C080E2F7FC8DE290E0B3010E94DC05A9
:100B200006C080E390E0B3010E94DC059A94D914DA
:100B3000C0F3DA94F101ED0DF11D808190E0B30175
:100B40000E94DC05DD20A9F706C080E290E0B30139
:100B50000E94DC05EA94EE20C1F743CEF3016681E2
:100B60007781CB012B96E2E10C940025FC010590E6
:100B7000615070400110D8F7809590958E0F9F1F9F
:100B80000895FC016150704001900110D8F78095E4
:100B900090958E0F9F1F0895DC01FC01672F7191C6
:100BA0007723E1F7329704C07C916D937083629153
:100BB000AE17BF07C8F308950F931F93CF93DF932A
:100BC0008C01EB018B8181FF1BC082FF0DC02E8148
:100BD0003F818C819D812817390764F4E881F98170
:100BE0000193F983E88306C0E885F985802F09958C
:100BF000892B31F48E819F8101969F838E8302C061
:100C00000FEF1FEFC801DF91CF911F910F91089552
:100C1000FA01AA27283051F1203181F1E8946F932D
:100C20006E7F6E5F7F4F8F4F9F4FAF4FB1E03ED0D3
:100C3000B4E03CD0670F781F891F9A1FA11D680F71
:100C4000791F8A1F911DA11D6A0F711D811D911DA4
:100C5000A11D20D009F468943F912AE0269F112419
:100C60003019305D3193DEF6CF010895462F47707D
:100C7000405D4193B3E00FD0C9F7F6CF462F4F70D8
:100C8000405D4A3318F0495D31FD4052419302D036
:100C9000A9F7EACFB4E0A6959795879577956795DC
:100CA000BA95C9F700976105710508959B01AC01DC
:100CB0000A2E06945795479537952795BA95C9F703
:100CC000620F731F841F951FA01D0895DC011296EB
:100CD0002C91129717968C9117972817D8F5ED91AC
:100CE000FC911197E20FF11D862F992787FD9095B2
:100CF00016960C90169702C0880F991F0A94E2F777
:100D00002081282B208313968C9113978F5F139645
:100D10008C93139716962C91169714963C911497D2
:100D2000822F90E0831B910997FD04C0231B169628
:100D30002C93089587E016968C93169712968C91B3
:100D400012978F5F12968C931297ED91FC91E80F9A
:100D5000F11D10820895FC018781681738F4019015
:100D6000F081E02DE60FF11D808108958FEF089549
:100D7000DC0117968C911797882369F090E0ED912C
:100D8000FC911197E90FF11D10829F5F17968C91CE
:100D900017979817A0F312961C92129713961C920D
:100DA000139787E016968C930895FC0180819181BA
:100DB0000E945B010895CF93DF93EC01842F6C8335
:100DC0001D824F8390E061E070E00E94950088836F
:100DD0009983CE010E94B8068C8147E050E0481B01
:100DE000510947305105A1F037E087E090E02D81AF
:100DF00061E070E0FB0102C0EE0FFF1F8A95E2F791
:100E00002E2B2D833150832F90E04817590794F3F0
:100E1000DF91CF910895FC0112A2A185B2850384D0
:100E2000F485E02D208131818D919C9111979183E2
:100E300080832D933C93DB018D919C9191838083E2
:100E400008957F928F929F92AF92BF92CF92DF923E
:100E5000EF92FF920F931F93CF93DF938C017B014F
:100E6000FC0171A0772021F1FB01608171814C01AF
:100E7000C0E0D0E021E0A22EB12C5C2F16161706A0
:100E800084F4F801C584D684F70122813381F4010A
:100E900083899489281B390B37FD49C0C216D306B4
:100EA0004CF4219682E090E0880E991EC71528F335
:100EB0008FEF2FC06130710559F141E006C0CE16A9
:100EC000DF067CF32617370719F14F5F242F30E038
:100ED0006217730734F3F901EE0FFF1FEE0DFF1DCC
:100EE000D901AC0FBD1FAA19BB09AA0FBB1FA00FC8
:100EF000B11F0190F081E02D53968D919C915497F4
:100F0000E81BF90BF7FFDBCFF095E195FF4FD7CF4B
:100F1000852FDF91CF911F910F91FF90EF90DF9080
:100F2000CF90BF90AF909F908F907F900895309515
:100F300021953F4FB3CF089508950895FC01838113
:100F4000948108952F923F924F925F926F927F9279
:100F50008F929F92AF92BF92CF92DF92EF92FF92C9
:100F60000F931F93DF93CF9300D000D0CDB7DEB7A0
:100F70005C01DC0113968D919C9114970197E1F02F
:100F80008FEFD50193968C9380E00F900F900F9088
:100F90000F90CF91DF911F910F91FF90EF90DF9015
:100FA000CF90BF90AF909F908F907F906F905F9009
:100FB0004F903F902F90089591968C91815087FD8E
:100FC000DFCF882E992487FC9094F401EE0FFF1F49
:100FD0007396EA0DFB1DFC83EB8328E131E0820E62
:100FE000931E6501C80CD91CA8EEBEEF8A0E9B1E8D
:100FF000482F00E010E075E1272E71E0372E2A0C13
:101000003B1CF501B596FA83E9830DC04150EB8195
:10101000FC813297FC83EB830894C108D10801500E
:10102000104047FDADCF2801480C591CAB81BC8155
:101030002D913C91121613064CF3EE24FF24E21A74
:10104000F30AB9E6EB16B2E4FB060CF048C0F50172
:101050008281682E772467FC7094F301EE0FFF1FE6
:10106000EA0DFB1D0388F489E02D2E273F2737FF6B
:10107000CDCFEE0FFF1FEE0FFF1FEE0FFF1FEE167F
:10108000FF0624F2F6018081873008F0BFCFD1013E
:101090003C91332309F4BACFE981FA8120E004C0FE
:1010A0002F5F3196231750F4818190E084159505C8
:1010B000B9F7808190E08615970591F7231709F419
:1010C000A5CFF50143A382E090E0948383838EE172
:1010D00091E0A80EB91ED5012C9381E056CFD50121
:1010E00012968C91682E772467FC7094F301EE0FB2
:1010F000FF1FEA0DFB1D0388F489E02DC701BF0126
:101100000E94A924683271050CF080CFAECF2F92D7
:101110003F924F925F926F927F928F929F92AF9287
:10112000BF92CF92DF92EF92FF920F931F93DF93C4
:10113000CF9300D000D00F92CDB7DEB71C018FEF58
:10114000F1018283F1A1F983FF2309F4BDC018E105
:10115000412E11E0512E420C531C4101AA24AA94A5
:10116000BA2CCC24DD2491012B5E3E4F3B832A8395
:101170003FEFA3163FEFB30609F452C03601F40166
:101180000388F489E02DFD83EC83F7FD77C0F5013A
:10119000EE0FFF1FE20DF31D838994892C813D81A1
:1011A000281739070CF06AC0F101EC0DFD1DE85E4F
:1011B000FE4F608170E0882777FD8095982F0E9410
:1011C0005F237B018C01EA81FB81608170E08827CD
:1011D00077FD8095982F0E945F232BE734E14EE244
:1011E0005EE30E9413249B01AC01C801B7010E9479
:1011F0000F2418160CF042C00894C11CD11C08948E
:10120000411C511C22E030E0820E931E3981C3162E
:10121000B8F553013FEFA3163FEFB30609F0AECF89
:101220003601F4010388F489E02DFD83EC83F7FD9A
:1012300025C0F201608170E0882777FD8095982FA6
:101240000E945F237B018C01EA81FB81608170E059
:10125000882777FD8095982F0E945F232BE734E144
:101260004EE25EE30E9413249B01AC01C801B7016A
:101270000E940F2418160CF4BFCF89CF3501BCCFC4
:101280008FEF68168FEF7806F9F0F101628281E046
:1012900090E09483838381E00F900F900F900F90E4
:1012A0000F90CF91DF911F910F91FF90EF90DF9002
:1012B000CF90BF90AF909F908F907F906F905F90F6
:1012C0004F903F902F90089580E0E6CFDC01A85E1C
:1012D000BE4F1D921D921D921D921D921C92AD51EA
:1012E000B140442399F4AB5EBE4F4C91A551B1403F
:1012F0000DC0FD01E60FF11D85A1FD01E80FF11DF7
:10130000E85EFE4F80818F5F80836F5F641788F394
:1013100008952F923F924F925F926F927F928F9299
:101320009F92AF92BF92CF92DF92EF92FF920F9374
:101330001F93DF93CF9300D00F92CDB7DEB79B837F
:101340008A8360E040E00E9466095524EA81FB81BF
:1013500041A035E1832E31E0932E8E0E9F1E541452
:1013600008F08EC0F52DFF5FF983F41508F084C0F6
:10137000852D90E04F2F5C01AA0CBB1CEA81FB81FC
:1013800025843684AE0EBF1E23E130E0A20EB31ECC
:101390003F01680E791E68E171E0660E771EA42F8A
:1013A000B0E06D01CC0CDD1CEA81FB81EC0DFD1D74
:1013B00023893489F501E080F180C9018E199F09E4
:1013C00097FD74C0281639060CF452C0F4018081D0
:1013D0008823E9F090E005C09F5FF40180819817B1
:1013E00068F4EA81FB81E90FF11D85A18417A1F75B
:1013F00055A29F5FF4018081981798F3F501E08072
:10140000F180EA81FB81EC0DFD1D23893489F30114
:101410008081E82FF0E06A817B81A60FB71FA85E6C
:10142000BE4F8C9190E08C010E0F1F1FBC01269FB8
:10143000C001279F900D369F900D1124B8010E9486
:10144000A9249B01EE9EC001EF9E900DFE9E900D83
:101450001124B8010E94A924260F371FF5013183FA
:1014600020832A813B81C20ED31EF601148A138A7F
:101470004F5F441508F493CF5980541408F472CF89
:101480000F900F900F90CF91DF911F910F91FF90D0
:10149000EF90DF90CF90BF90AF909F908F907F9014
:1014A0006F905F904F903F902F9008959095819509
:1014B0009F4F88CFCF93DF93EC010E948909CE0123
:1014C00060E040E00E946609CB5EDE4F8881C55136
:1014D000D140883230F0CE010E948708CE010E94B0
:1014E000A207DF91CF910895DC01ED91FC9101906D
:1014F000F081E02D099508956F927F929F92AF92AF
:10150000BF92CF92DF92EF920F93DF93CF9300D0F1
:1015100000D0CDB7DEB76C01FC0162807380F301AF
:1015200081A1843008F495C085E191E0680E791EB0
:10153000F30160818BEE9EEF680E791E70E08827C4
:1015400077FD8095982F0E945F2329E23CE54FE0CC
:101550005EE30E9413240E943123762FAA24AA94CA
:10156000BA2C00E0992460E030E0A32FB0E0F30152
:10157000EA0FFB1FE85EFE4FE080E716C8F1AA0FF6
:10158000BB1FA60DB71D53964D915C915497141631
:1015900015060CF078C0F60125812F3F09F46AC0CA
:1015A000E22FFF27E7FDF095EE0FFF1FE60DF71D79
:1015B00083899489841795070CF45CC0F601258310
:1015C00027812F3F09F45DC0E22FFF27E7FDF0954B
:1015D000EE0FFF1FE60DF71D838994894817590701
:1015E0000CF44FC06E0D0F5FA40EB51EF6012783DD
:1015F0003F5FF30181A1381708F4B7CF70E0882767
:1016000077FD8095982F0E945F2369837A838B836F
:101610009C8385E191E0680E791EF301608170E0A2
:10162000882777FD8095982F0E945F232AE037ED69
:1016300043EA5CE30E9413249B01AC0169817A8137
:101640008B819C810E940F2418161CF0091509F447
:1016500045C080E00F900F900F900F90CF91DF91D9
:101660000F91EF90DF90CF90BF90AF909F907F90C1
:101670006F900895232FF601258327812F3F09F0CE
:10168000A3CF232FAFCFF60124812F3F29F1E22FE3
:10169000FF27E7FDF095EE0FFF1FE60DF71D83898D
:1016A000948948175907C4F0F601248326812F3FF7
:1016B00069F0E22FFF27E7FDF095EE0FFF1FE60D23
:1016C000F71D83899489841795070CF4232F6E19CD
:1016D0009394F60126838CCF232FE6CFC50163E0D8
:1016E00070E00E94A924F6017187608794819F3F72
:1016F00009F4AFCF86818F3F09F4ABCF981709F477
:10170000A8CF25812F3F09F4A4CF97819F3F09F4EB
:10171000A0CF80E0291709F49DCF81E09BCF8F9265
:101720009F92AF92BF92CF92DF92EF92FF921F9360
:10173000DF93CF9300D00F92CDB7DEB77C016B0162
:101740005E010894A11CB11CD501E9E0F1E083E041
:1017500001900D928150E1F7D701ED91FC916281EA
:1017600083E0689FB0011124C6010E942721C114A3
:10177000D10489F1D701ED91FC9110E084E0882E2D
:1017800081E0982ECF01612F0E94AB0600D000D0DF
:1017900000D0EDB7FEB73196ADB7BEB71296BC928A
:1017A000AE92119793828282848315820E94B50340
:1017B0008DB79EB706960FB6F8949EBF0FBE8DBF2D
:1017C000C601B5010E94E0211F5FD701ED91FC9198
:1017D00082818117B8F60F900F900F90CF91DF9113
:1017E0001F91FF90EF90DF90CF90BF90AF909F90B0
:1017F0008F900895FC018FEF848385838683878390
:1018000084E18287808191810E94B80608950F93B8
:101810001F938C01FC0111A2148213828FEF82832B
:10182000878D90A10E94B806F80116861586148A45
:10183000138A168A158A108E178A128E118E148EAC
:10184000138E168E158E1F910F910895CF93DF93EF
:10185000EC010E94070CCB5EDE4F1882C551D140CF
:1018600019A21CA21C821B828FEF8BA38A83FE010C
:10187000DE01A85EBE4F80E0148A138A1D928F5F3E
:1018800032968630C9F71AA286E990E09E878D8746
:101890008AE999E9A9E9BEE38F87988BA98BBA8B6E
:1018A000C25EDE4F1882289719921882DF91CF917D
:1018B0000895EF92FF920F931F938C01FC017383A5
:1018C000628388E090E00E943E1CF82EE92E61E0E1
:1018D0004EE10E94DB06F801F082E182C8010E941D
:1018E000FA0B1F910F91FF90EF900895EF92FF92E6
:1018F0000F931F938C0183E392E0F801918380831F
:1019000088E090E00E943E1CF82EE92E62E041E063
:101910000E94DB06F801F78EE0A21086178216827D
:101920001582C801059692878187C801079694871A
:10193000838712A2C8010E94070C1F910F91FF908C
:10194000EF9008950F931F938C010E94760C87E20D
:1019500092E0F801918380831682158210861782A7
:10196000C801059692878187C80107969487838767
:101970008FEF83A3C8010E94260C1F910F91089539
:10198000AF92BF92CF92DF92EF92FF920F931F938D
:101990008C010E94A20C8BE192E0F801918380837C
:1019A00060E7A62E61E0B62EA00EB11E50E0E52E37
:1019B00051E0F52EC501B7010E942B2247E7C42E46
:1019C00041E0D42EC00ED11EC601B7010E942B22C9
:1019D000C50166E470E00E942721C60164E170E061
:1019E0000E94272101591E4FF80110821F910F916B
:1019F000FF90EF90DF90CF90BF90AF900895FF924F
:101A00000F931F93CF93DF938C01DC011296CD913E
:101A1000DC911397DE01AB5EBE4F8C91882309F4F5
:101A200000C1FF2460E056C04F2D50E0DE01A40F3E
:101A3000B51F95968C919597282F30E0F8018481F9
:101A4000992787FD90952817390709F475C0858176
:101A5000992787FD90952817390709F46DC0F8017B
:101A60008681682F772767FD70952617370709F459
:101A700093C0F8018781992787FD9095281739072A
:101A800009F48AC0CB5EDE4F8881E82FF0E0D801F0
:101A90001A962C91E21BF1094E175F070CF0B1C0AA
:101AA000F801808191810E94B806D8011296ED91CB
:101AB000FC911397E25EFE4FF08261E01296CD91A9
:101AC000DC911397F394DE01AB5EBE4F9C91F91647
:101AD00008F04DC0662309F0A7CF4F2D50E0FE015E
:101AE000E40FF51F85A1282F30E0F80184819927A4
:101AF00087FD909528173907C1F08581992787FDC3
:101B000090952817390789F0F8018681992787FD74
:101B100090952817390749F0D80117968C91992785
:101B200087FD90952817390769F6C25EDE4FF88267
:101B3000F801C281D3817ACFD8014D915C9160E0E8
:101B4000220F331FC20FD31F8B899C8997FF61E03F
:101B5000CA010E94660661E0F801C281D381F39454
:101B6000DE01AB5EBE4F9C91F91608F4B3CFF916B7
:101B700009F458C030E0D801ED91FC9111979381A0
:101B80001A968C91981708F044C0832FDF91CF915B
:101B90001F910F91FF900895CB5EDE4F8881C55154
:101BA000D140E82FF0E0CF010197481759070CF01A
:101BB0006ECF96968C91282F30E06217730751F004
:101BC000D80117968C91992787FD9095281739078A
:101BD00009F05DCFF8014081518160E0220F331F91
:101BE000C20FD31F8B899C8997FF61E0CA010E94B5
:101BF0006606F39461E0D8011296CD91DC911397BB
:101C000061CF30E0D801ED91FC918381821708F417
:101C1000BCCF31E0832FDF91CF911F910F91FF90C7
:101C2000089590E0C25EDE4F8881823008F4A2CF32
:101C3000981B9C93D8011296ED91FC911397E25E4C
:101C4000FE4F6081EE51F14070E06B5D7F4F6E0F93
:101C50007F1FEB5EFE4F408150E04F5F5F4FCF0133
:101C6000805F90400E94DB02D8011296ED91FC91BA
:101C70001397EA5EFE4F81E080837CCFCF92DF92A4
:101C8000EF92FF920F931F93DF93CF9300D000D07A
:101C9000CDB7DEB78C0135E1C32E31E0D32EC80EAF
:101CA000D91ED6018C9190E08F3E91050CF0FAC0C0
:101CB000D80194961C92949719960D90BC91A02DE2
:101CC0002D913C911197F80183859485FC016081E9
:101CD0007181F601408190915602F80181A1891726
:101CE00010F4F80191A3442309F4CDC0EE2480E060
:101CF00090E06227732777FD13C120E030E04F3E6C
:101D000011F021E030E082239323892B09F0C7C032
:101D100081E090E09A8389831C821B828D919C9143
:101D20009C838B83C801BE016F5F7F4F0E94210798
:101D3000F82E87FD04C1F6018081F801E80FF11D3E
:101D4000F5A2823020F084A18F1509F4F1C0EF2DA7
:101D5000FF27E7FDF095EE0FFF1FE00FF11F2B812E
:101D60003C8183899489280F391F37FDE5C035955B
:101D70002795348B238BD6018C918F5F8C93FF2416
:101D8000EE2009F46CC0F6018081883238F083E0DF
:101D900090E0D80114969C938E931397FF2009F43A
:101DA00045C0F601F080AF2DB0E0BD01615070403C
:101DB000FFEF6F3F7F0709F49CC050915602F80176
:101DC000E60FF71F85A1851709F482C09396F801E5
:101DD000EA0FFB1F20E030E0959707C080812F5F5E
:101DE0003F4F3197851709F473C061507040CD01A2
:101DF000821B930B8F5F9F4F89F7E52FF0E0EE0F6B
:101E0000FF1FE00FF11F8B819C81948B838BD60188
:101E10008C91F801E80FF11D55A38F5F8C93E52F8E
:101E2000EF5FE0935602E63009F466C00F900F9022
:101E30000F900F90CF91DF911F910F91FF90EF9036
:101E4000DF90CF90089550915602E50FF11DE85EA6
:101E5000FE4F8081823008F47CC0EE24FF24D6013E
:101E60008C91883208F04EC0EE2009F097CFC8015F
:101E70000E94260CD80192961C9210925602FF20C6
:101E800009F08FCFD3CFD80191961C9291971092E1
:101E90005602EE2419960D90BC91A02D39CFEE2458
:101EA000E39436CF095E1E4F81E0F801808307512D
:101EB0001140D801ED91FC910680F781E02DC80119
:101EC00009950A5E1E4FF801108206511140F0CEAE
:101ED0006F5F7F4F4F2D461BD6014C936B5D7F4F3D
:101EE000600F711F50E04F5F5F4FC80185960E94E1
:101EF000DB025091560281CF10925602D801919682
:101F0000EC9394CF81E0F80182A30190F081E02D61
:101F10000680F781E02DC80109951092560286CF00
:101F200081E090E020E030E04F3E09F0EACEEBCED9
:101F3000C8010E94260C0BCF2F5F3F4F18CFC8015E
:101F400060E040E00E946609F80181A1863009F452
:101F50007ACFFF24F39414CF0F931F93CF93DF9383
:101F60008C01DC0192961C92929719960D90BC916F
:101F7000A02DEC01EB85FC85208131818D919C9118
:101F80001197918380832D933C93DB018D919C91DC
:101F900091838083C8010E943E0E8AA1DF91CF9178
:101FA0001F910F9108950F931F93CF93DF938C018F
:101FB000EB01CB0167E070E00E942721209779F0C8
:101FC000CE016EE071E00E94E021F801608571852C
:101FD000CE010E947021CE016BE30E94CD21DF91E2
:101FE000CF911F910F9108950F931F93CF93DF937C
:101FF0008C01EB01CB0160E270E00E942721209769
:1020000009F470C0CE0161E171E00E94E021D801C5
:102010001296ED91FC91139714968C91992787FD58
:102020009095880F991FE80FF91F63897489CE0175
:102030000E947021CE016BE30E94CD21CE0165E1AB
:1020400071E00E94E021D8011296ED91FC91139766
:1020500015968C91992787FD9095880F991FE80F09
:10206000F91F63897489CE010E947021CE016BE350
:102070000E94CD21CE0169E171E00E94E021D801EA
:102080001296ED91FC91139716968C91992787FDE6
:102090009095880F991FE80FF91F63897489CE0105
:1020A0000E947021CE016BE30E94CD21CE016DE133
:1020B00071E00E94E021D8011296ED91FC911397F6
:1020C00017968C91992787FD9095880F991FE80F97
:1020D000F91F63897489CE010E947021CE016BE3E0
:1020E0000E94CD21DF91CF911F910F910895CF9341
:1020F000DF93FC01C081D181209731F0CE010E9495
:10210000D506CE010E943B1CDF91CF910895CF925E
:10211000DF92EF92FF920F931F937A01690101E220
:1021200015E0C8010E94DF1DC801B7010E94DF1D34
:10213000C801B6010E94DF1D1F910F91FF90EF9023
:10214000DF90CF900895AF92BF92DF92EF92FF920F
:102150000F931F93CF93DF93EC01F62ED42E5801EB
:1021600081E295E0B9010E94DF1DDF1458F1EE24F1
:102170008E010F0D111D81E295E0F80165A14AE085
:1021800050E00E94451DF80185A1E82688E09CE802
:10219000E0FAE6940EF4E9268A95D1F7F394DF1479
:1021A00038F71E2D81E295E0B5010E94DF1D812FD9
:1021B000DF91CF911F910F91FF90EF90DF90BF9033
:1021C000AF90089510E0EECF2F923F924F925F9222
:1021D0006F927F928F929F92AF92BF92CF92DF9237
:1021E000EF92FF920F931F93DF93CF93CDB7DEB79C
:1021F00062970FB6F894DEBF0FBECDBF7C018C0195
:102200000B5E1E4FF80180818832C8F462960FB6CB
:10221000F894DEBF0FBECDBFCF91DF911F910F911C
:10222000FF90EF90DF90CF90BF90AF909F908F90F6
:102230007F906F905F904F903F902F9008955E2C0D
:102240004F2CC7010E945A0AF70183819481823082
:10225000910509F47EC0019779F0F70112A226E1F9
:1022600031E0E20EF31EF7018081882379F6852D97
:10227000942D0E94260CCACFF8018081883268F321
:10228000B0E78B2EB1E09B2E8E0C9F1CC40160E04A
:1022900071E00E944522A7E76A2EA1E07A2E6E0C1B
:1022A0007F1CC30160E071E00E944522C40162E02E
:1022B0000E94CD21F8E02F2E312C2C0E3D1EC101A5
:1022C000B7010E94590CC1010E94FA0BC1010E9482
:1022D0007C0A882309F0A1C1C4016DE371E00E946A
:1022E000E021C4016BE30E94CD21F70191A1992364
:1022F00009F434C1BB2404C0B394B91608F02EC14C
:10230000CB2CDD24F701EC0DFD1DE85EFE4F808136
:10231000882391F3C4016BE371E00E94E021C401C2
:102320006B2D0E94A121C40164E271E00E94E021B2
:10233000CC0CDD1CCE0CDF1CF60163897489C40152
:102340000E947021C4016BE30E94CD21F70191A18D
:10235000D3CF3EE1632E31E0732E6E0C7F1CF30170
:102360006081462F4E5FF7018281A82FBB27A7FD12
:10237000B095F801508104C04E5F451708F07BC04E
:10238000F701E40FF11D85A190E08A179B07A1F7E3
:1023900026A130E0F70183A1992787FD90952817A2
:1023A000390751F7C42ECA945C1508F4C52E852D43
:1023B000942D4C2D0E9466098C2D90E0F301208114
:1023C000821B910988970CF46DC020E7A22E21E0B2
:1023D000B22EAE0CBF1CC50160E071E00E94452228
:1023E00097E7892E91E0992E8E0C9F1CC40160E026
:1023F00071E00E944522C50162E00E94CD21C50125
:1024000061E271E00E94E021C5016BE30E94CD21F1
:10241000F70191A1992309F44CC0DD2404C0D394A1
:10242000D91608F046C00D2D10E0F701E00FF11F9E
:10243000E85EFE4F8081882391F3C50160E50E942C
:10244000CD21C5016D2D0E94A121C50164E271E07D
:102450000E94E021000F111F0E0D1F1DF80163895E
:102460007489C5010E947021C5016BE30E94CD21D2
:10247000F70191A1D4CFC42E5417C8F0852D942D07
:102480004C2D0E946609F8018081803F08F49DCFA1
:10249000F3018081823030F08C2D90E08F3E9105E9
:1024A0000CF09AC0852D942D0E94260CD8CEC52EF6
:1024B000E5CFC50166E271E00E94E021C4016BE353
:1024C0000E94CD21C40169E271E00E94E021F70180
:1024D0006281772767FD7095C4010E947021C40155
:1024E0006BE30E94CD21C4016DE271E00E94E02106
:1024F000F70163A1772767FD7095C4010E947021E1
:10250000C4016BE30E94CD2127E131E0E20EF31E0E
:10251000F701808129EE3EEFE20EF31E8823A1F43D
:10252000C40163E00E94CD21C4016AE00E94CD2174
:10253000C701F30160814C2D950184010E94A31015
:1025400081E0F70182A38BCEC40161E371E00E94B8
:10255000E021C4016BE30E94CD21E2CFC40166E219
:1025600071E00E94E021C3016BE30E94CD21C30111
:1025700069E271E00E94E021F7016281772767FD3F
:102580007095C3010E947021C3016BE30E94CD21AD
:1025900027E131E0E20EF31EF701808129EE3EEFE4
:1025A000E20EF31E882309F076C0C30163E00E94A7
:1025B000CD21C3016AE00E94CD21C70160E0F8018E
:1025C0004081940183010E94A31081E0F70182A35E
:1025D000C1010E94771043CE81E295E063E371E090
:1025E0000E94C91DF8014081F3016081461BF8017A
:1025F000408370E06B5D7F4F6E0D7F1D50E04F5F3D
:102600005F4FC70185960E94DB0226E131E0E20EB2
:10261000F31E81E0F7018083F9CDC1010E94FF0C18
:10262000882309F459CE8E010F5F1F4FC80160E067
:1026300071E00E942B22C80166E271E00E944522EF
:10264000C101B8010E948F0BC40168E371E00E94D0
:10265000E021C4016BE30E94CD21C101B4010E94BD
:10266000F40FC3016BE30E94CD21C101B3010E94AD
:10267000D30FC30163E00E94CD21C3016AE00E9431
:10268000CD21C701B401A80193010E948710C801A0
:102690000E942B239ACFC30161E371E00E94E021E5
:1026A000C3016BE30E94CD2180CF1F920F920FB622
:1026B0000F9211242F933F934F935F936F937F93C8
:1026C0008F939F93AF93BF93EF93FF93E0915A0241
:1026D000F0915B020995FF91EF91BF91AF919F91AE
:1026E0008F917F916F915F914F913F912F910F90BB
:1026F0000FBE0F901F9018958130910531F0892BF6
:1027000019F46F5F7F4FE1F008956F5F7F4FE1F73E
:1027100080E580935C0210925D0280915D0280935F
:102720005F0280915F0280935E0281E093E062EB42
:1027300071E00E942B2289E093E00E94C00C089572
:102740008BE192E090930A038093090380E894E080
:102750000E942B2389E794E00E942B2381E093E0E1
:102760000E942B23089580E090E06FEF7FEF0E949E
:102770007C13089581E090E06FEF7FEF0E947C135F
:102780000895FF920F931F93CF93DF93F82E01E2EA
:1027900015E0C80163EB71E00E94C91DC8016F2DEF
:1027A0004AE050E00E94451DC8016EEB71E00E94B6
:1027B000C91DCF2DD0E0CC0FDD1FCC0FDD1FCC0FFE
:1027C000DD1FFE01E55DFB4F60817181C8014AE0BC
:1027D00050E00E94971DC80162EC71E00E94C91D83
:1027E000C65DDB4F6881772767FD7095C8014AE0B9
:1027F00050E00E94971DC80167EC71E00E94CC1D5B
:10280000DF91CF911F910F91FF900895AF92BF92EA
:10281000CF92DF92EF92FF920F931F93DF93CF93AC
:10282000CDB7DEB762970FB6F894DEBF0FBECDBF4F
:102830008E01075F1F4F81E093E0B8014AE050E04E
:1028400023E030E00E94E020C80167EC71E00E94C4
:10285000CD020E948802D82E5E010894A11CB11CF2
:10286000D501EBE3F2E088E001900D928150E1F7B1
:1028700081E093E061E070E00E946C20813409F413
:102880003EC00D2D10E0EE24FF24CC2481E093E027
:1028900061E070E00E946C208235F1F08D2D0E9485
:1028A000C1138091780490E00196801791071CF481
:1028B000D394D092780462960FB6F894DEBF0FBE20
:1028C000CDBFCF91DF911F910F91FF90EF90DF90DF
:1028D000CF90BF90AF900895CB82FD82EC82F8013B
:1028E000EE0FFF1FEE0FFF1FEE0FFF1FE85DFB4F08
:1028F000D50188E00D9001928150E1F7CFCF80E0C3
:1029000090E067EC71E00E94CD020E948802C82E20
:1029100080E090E067EC71E00E94CD020E948802A6
:102920007C010D2D10E0CB829D838C83F801EE0F8E
:10293000FF1FEE0FFF1FEE0FFF1FE85DFB4FD501DE
:1029400088E00D9001928150E1F7A0CF0E94FE1E19
:102950009B01AC018091870490918804A091890427
:10296000B0918A04281739074A075B0748F4809119
:102970008B0490918C04019690938C0480938B042B
:1029800020938704309388044093890450938A04E9
:10299000CA01B90128EE33E040E050E00E94BC24B7
:1029A000C90108951F9311E081E295E00E941E1B6A
:1029B000892BA9F081E295E00E944F1B682F8A3095
:1029C000A1F08B3074F4882381F081E093E00E94C1
:1029D000CD2181E295E00E941E1B892B59F71F91A2
:1029E00008958D3011F0833281F710930803DCCF06
:1029F000609100038DE00E94092010920003089569
:102A0000EF92FF921F93CF93DF937C0181E093E0DD
:102A100064E40E94DB20182F1F5F612F70E080911B
:102A200005039091060386179707A8F42FC068EE58
:102A300073E00E94A924882777FD8095982F0E9433
:102A4000321F1F5F612F70E0809105039091060394
:102A500086179707D8F081E093E00E946C20C82F7A
:102A6000D0E0CC0FDD1FCE0DDF1D60E088819981A5
:102A700097FF61E08BE00E940920888199812FE116
:102A800081349207A4F60E94581FDBCFDF91CF91CB
:102A90001F91FF90EF900895EF92FF920F931F9375
:102AA000082FE62E8BE061E00E94092010E0809163
:102AB0001502909116029C01029FC001039F900D88
:102AC000129F900D11240E94581F8BE060E00E941D
:102AD0000920FF2480911502909116029C01E29E2C
:102AE000C001E39E900DF29E900D11240E94581F8C
:102AF0001F910F91FF90EF90089580E00E94491E72
:102B0000089580E069EF78E141E050E00E94261EE0
:102B1000089581E093E061E070E00E946C208135CF
:102B200061F081E093E061E070E00E946C20853408
:102B300009F008950E94811508950E947D15F1CF36
:102B40002F923F924F925F926F927F928F929F92BD
:102B5000BF92CF92DF92EF92FF920F931F93DF937A
:102B6000CF93CDB7DEB7ED970FB6F894DEBF0FBEAB
:102B7000CDBF81E093E061E070E00E946C2082357F
:102B8000C1F0ED960FB6F894DEBF0FBECDBFCF916A
:102B9000DF911F910F91FF90EF90DF90CF90BF904A
:102BA0009F908F907F906F905F904F903F902F906D
:102BB00008956E010894C11CD11CC60162EB71E03E
:102BC0000E942B228E01085F1F4FC80167EC71E045
:102BD0000E942B2281E093E0B80142E050E00E9485
:102BE0009F20F82EC8010E942B23BB248FE0682E63
:102BF000712C6C0E7D1E06E1802E912C8C0E9D1E7C
:102C00001DE1412E512C4C0E5D1EB4E22B2E312CB9
:102C10002C0E3D1EEF2CFF24E7FCF09487010F5F84
:102C20001F4F81E093E0B8010E946C20843409F4C6
:102C300058C081E093E064E40E94DB200817190784
:102C40000CF04FC0C30167EC71E00E942B2282E0C0
:102C500090E0E80EF91E81E093E0B301A7010E9425
:102C60009F20F82EC3010E942B232F2D332727FDF1
:102C7000309521503040C40161E073E0A8010E940A
:102C8000C122C601B4010E941423C4010E942B2357
:102C9000C60160E070E00E946C20803509F443C0FA
:102CA000C60160E070E00E946C20823509F0B2CF6E
:102CB000C60162E070E00E946C208D3309F0AACF5B
:102CC000CE018B96B60142E050E00E940823CE016F
:102CD0008B960E948E20B62ECE018B960E942B23BF
:102CE00099CF0E947D15BB2091F000E052E3E52EC4
:102CF000F12CEC0EFD1EC7010E94001562E070E091
:102D000080E090E00E94321F0F5F0B15A0F30E943D
:102D1000811581E295E061E073E00E94121EC60118
:102D20000E942B232ECFC60162E070E00E946C202F
:102D30008D3309F0B5CFC201B60141E050E021E08A
:102D400030E00E94C122C2010E948E20162FC201D3
:102D50000E942B23C101B60143E050E00E940823EA
:102D6000C1010E948E20E12FF0E0EE0FFF1FEC0D5D
:102D7000FD1D72AB61ABC1010E942B234BCFEF92C3
:102D8000FF920F931F93CF93DF937C010E947D15D9
:102D900080911402882391F100E010E081E06FE15E
:102DA0000E944C15F7018081882301F1E70110C0D2
:102DB000863469F1803341F481E063E00E944C1570
:102DC00081E063E00E944C1589812196882371F08F
:102DD000813371F783E061E00E944C1583E061E08C
:102DE0000E944C1589812196882391F70F5F1F4F10
:102DF0008091140290E00817190784F20E9481154F
:102E0000DF91CF911F910F91FF90EF90089581E096
:102E100063E00E944C1583E061E00E944C15D4CF22
:102E2000EF92FF920F931F93DF93CF93CDB7DEB74F
:102E3000EA970FB6F894DEBF0FBECDBF81E093E0F6
:102E400061E070E00E946C20843709F44EC081E09C
:102E500093E061E070E00E946C20823741F181E0F4
:102E600093E061E070E00E946C20833709F444C075
:102E700081E093E061E070E00E946C20833609F409
:102E800067C081E093E061E070E00E946C208037D1
:102E900009F479C0EA960FB6F894DEBF0FBECDBF35
:102EA000CF91DF911F910F91FF90EF9008958E01C8
:102EB0000C5F1F4FC80161E073E042E050E00E94E8
:102EC0000823C8017E010894E11CF11CB70143E00E
:102ED00050E020E030E00E94E020C8010E942B2357
:102EE000C7010E9488028093140281E295E061E0AC
:102EF00073E00E94121ECECF8DE061E00E94092097
:102F00008E01055F1F4FC80161E073E042E050E0B1
:102F10000E9408232EE2E22EF12CEC0EFD1EC801C9
:102F2000B7014DE050E020E030E00E94E020C80111
:102F30000E942B23C7010E94BF168DE060E00E9413
:102F4000092081E295E061E073E00E94121EA2CFA9
:102F50008E010E5E1F4FC80161E073E042E050E059
:102F60000E940823C8010E948E207093160260936D
:102F70001502C8010E942B2381E295E061E073E015
:102F80000E94121E87CF99E1E92EF12CEC0EFD1E56
:102F9000C70162EB71E00E942B22C70164E170E07F
:102FA0000E942721C70169EC71E00E9445228E0131
:102FB000005E1F4FC801609114024AE00E948F22F8
:102FC000C701B8010E94F021C8010E942B23C7014C
:102FD00064ED71E00E94E0218E01095D1F4F609158
:102FE000150270911602C8014AE00E945E22C701D4
:102FF000B8010E94F021C8010E942B2381E295E0D4
:10300000B7010E94121EC7010E942B2343CFDF93FA
:10301000CF9300D0CDB7DEB781E093E060E070E001
:103020000E946C208F3309F457C081E093E060E088
:1030300070E00E946C20863509F4AAC081E093E01C
:1030400060E070E00E946C208235B9F480915005F8
:1030500090915105009709F4B9C0BE016F5F7F4F91
:10306000681B790B81E295E04AE050E00E94AA1DBE
:103070000F900F90CF91DF91089581E093E060E091
:1030800070E00E946C20893609F48DC081E093E0E5
:1030900060E070E00E946C20833509F48EC081E00E
:1030A00093E060E070E00E946C20843709F491C0E6
:1030B00081E093E060E070E00E946C20883509F4C4
:1030C00095C081E093E060E070E00E946C2086345F
:1030D00079F60E940614CCCF81E295E06FE30E945E
:1030E0008E1C81E295E068E670E00E946B1C81E234
:1030F00095E066E50E948E1C81E295E060E20E9408
:103100008E1C81E295E069E60E948E1C81E295E0CA
:1031100060E20E948E1C81E295E062E50E948E1CB6
:1031200081E295E060E20E948E1C81E295E064E716
:103130000E948E1C81E295E060E20E948E1C81E27A
:1031400095E068E50E948E1C81E295E060E20E94B5
:103150008E1C81E295E066E40E948E1C81E295E07F
:1031600060E20E948E1C81E295E063E50E948E1C65
:1031700081E295E060E20E948E1C81E295E062EBC4
:1031800071E00E94CC1D0F900F90CF91DF910895B8
:1031900081E295E066ED71E00E94CC1D0F900F90EA
:1031A000CF91DF91089589E093E00E949E07892BDB
:1031B000D1F081E0809308035BCF89E093E00E9427
:1031C0009E07892BB1F70E94A01552CF84E595E0A8
:1031D00044CF0E94A614BC0181E295E04AE050E091
:1031E0000E94AA1D45CF0E94101742CF0E94891548
:1031F0003FCFEF92FF920F931F93CF93DF93809176
:103200008D04882309F45EC00E940C1F7B018C0191
:1032100082E00E943C209C0180919504909196044C
:10322000A0919704B0919804B801A701481B590BCD
:103230006A0B7B0BDB01CA01E0929504F0929604C5
:1032400000939704109398044A3551056105710560
:1032500084F181305DE7950750E0A50750E0B507A0
:103260007CF1C1E0DDE7232B19F0D095C195DF4F4C
:1032700080915D028035E8F480915D028F5F8093DC
:103280005D0280915E0260915C0290E070E00E94BD
:10329000952480935E02E0915E02F0E0EE0FFF1F46
:1032A000E05AFD4FD183C08380915E028F5F80938F
:1032B0005E02DF91CF911F910F91FF90EF900895E3
:1032C000EC01D1CF8DE894E00E942D1C892B09F4EC
:1032D0009BCF0E940C1F609395047093960480937B
:1032E0009704909398048DE894E00E94371C8CCF4B
:1032F000FF920F931F93DF93CF9300D0CDB7DEB72C
:10330000809108038823E1F58E010F5F1F4FFF2492
:10331000F39480915D02882359F180915D02815080
:1033200080935D0280915F0260915C0290E070E0AA
:103330000E94952480935F0280915F02E82FF0E065
:10334000EE0FFF1FE05AFD4F208131818F5F809388
:103350005F023A83298389E093E0B8010E94740AEE
:103360008823B9F2F092000380915D028823A9F6C8
:103370000F900F90CF91DF911F910F91FF900895C3
:10338000109208030E94071880910803882321F0F7
:1033900081E080930003B8CF81E093E062EB71E0BD
:1033A0000E944522F5CF81E295E040E051EE60E0D9
:1033B00070E00E94971A82E060E00E949D1F8BE0FF
:1033C00061E00E949D1F8DE061E00E949D1FE1E889
:1033D000F0E080E180831092800082E080935902C7
:1033E00088EA91E690935802809357029093870061
:1033F0008093860082E1808388EF94E190935B0262
:1034000080935A0281E080936F000E94811581E0D1
:1034100093E064E170E00E94272108951F920F92CB
:103420000FB60F9211242F933F934F938F939F9337
:10343000EF93FF938091C00082FD1DC04091C600B4
:103440002091D9043091DA042F5F3F4F2F733070F1
:103450008091DB049091DC042817390771F0E0912A
:10346000D904F091DA04E756FB4F40833093DA0435
:103470002093D90402C08091C600FF91EF919F91E3
:103480008F914F913F912F910F900FBE0F901F90F2
:103490001895E0912D05F0912E05E05CFF4F81918C
:1034A000919120813181821B930B8F739070892BB6
:1034B00011F00E94D21408951F920F920FB60F922E
:1034C00011242F933F938F939F93EF93FF9320911A
:1034D0001D0530911E0580911F059091200528172C
:1034E000390731F48091C1008F7D8093C10014C0F1
:1034F000E0911F05F0912005E352FB4F2081809160
:103500001F059091200501968F7390709093200570
:1035100080931F052093C600FF91EF919F918F919B
:103520003F912F910F900FBE0F901F901895AF9263
:10353000BF92DF92EF92FF920F931F93CF93DF938F
:10354000EC017A018B01DD24403081EE580780E0E8
:10355000680780E0780711F0DD24D39491E0A92E6C
:10356000B12CEC89FD89DD2069F0C50108A002C0FD
:10357000880F991F0A94E2F7808360E079E08DE379
:1035800090E005C0108260E874E88EE190E0A80148
:1035900097010E94BC242150304040405040569535
:1035A00047953795279580E12030380720F0DD20BA
:1035B00011F0DD24D6CFE889F9893083EA89FB89C7
:1035C000208319A2EE89FF89408121E030E0C90102
:1035D0000C8C02C0880F991F0A94E2F7482B408395
:1035E000EE89FF894081C9010D8C02C0880F991FA7
:1035F0000A94E2F7482B4083EE89FF894081C90194
:103600000E8C02C0880F991F0A94E2F7482B408362
:10361000EE89FF8980810F8C02C0220F331F0A942C
:10362000E2F7209528232083DF91CF911F910F91FE
:10363000FF90EF90DF90BF90AF900895DC011C9653
:10364000ED91FC911D97E05CFF4F219131918081BC
:103650009181281B390B2F733070C9010895DC014B
:103660001C96ED91FC911D97E05CFF4F208131810C
:10367000E054F040DF01AE5BBF4F8D919C911197FC
:103680002817390719F42FEF3FEF07C08D919C9150
:10369000E80FF91F8081282F30E0C9010895DC016F
:1036A0001C96ED91FC911D97E05CFF4F20813181CC
:1036B000E054F040DF01AE5BBF4F8D919C911197BC
:1036C0002817390719F42FEF3FEF10C08D919C9107
:1036D0001197E80FF91F20818D919C911197019608
:1036E0008F73907011969C938E9330E0C90108956A
:1036F000DC0191968C919197882339F05496ED9145
:10370000FC915597808186FFF9CF91961C92089580
:10371000CF93DF93EC01EE85FF85E05CFF4F2081C6
:103720003181E054F0402F5F3F4F2F733070DF0145
:10373000AE5BBF4F8D919C91119728173907D1F33C
:10374000E05CFF4F80819181E054F040E80FF91F69
:103750006083EE85FF85E05CFF4F31832083EE8937
:10376000FF89208181E090E00F8C02C0880F991FB3
:103770000A94E2F7282B208381E089A3EC89FD8954
:1037800080818064808381E090E0DF91CF91089513
:10379000109224051092230588EE93E0A0E0B0E09B
:1037A0008093250590932605A0932705B0932805BF
:1037B00087E492E0909322058093210589E994E0C3
:1037C00090932E0580932D058DED94E09093300518
:1037D00080932F0585EC90E090933205809331051E
:1037E00084EC90E0909334058093330580EC90E076
:1037F000909336058093350581EC90E090933805E1
:103800008093370582EC90E090933A0580933905D8
:1038100086EC90E090933C0580933B0584E0809398
:103820003D0583E080933E0587E080933F0585E07A
:103830008093400581E0809341050895CF93DF9305
:103840000E94621F0E94D319C9E4DAE10E9478192C
:103850002097E1F30E94491AF9CFFC0120E030E003
:103860008081882311F421E030E0C9010895FC0132
:1038700081E0808308950E945B0108950E94B10059
:103880000895CF92DF92EF92FF920F931F93CF9301
:10389000DF937C016B018A01C0E0D0E00FC0D6014C
:1038A0006D916D01D701ED91FC910190F081E02DBA
:1038B000C7010995C80FD91F015010400115110506
:1038C00071F7CE01DF91CF911F910F91FF90EF9093
:1038D000DF90CF900895EF92FF920F931F93CF93B5
:1038E000DF937C018B01C0E0D0E0F8010F5F1F4F38
:1038F0006491662359F0D701ED91FC910190F0811C
:10390000E02DC7010995C80FD91FEFCFCE01DF9178
:10391000CF911F910F91FF90EF900895DC01ED91F1
:10392000FC910190F081E02D09950895EF92FF92AE
:103930000F931F938C01DC01ED91FC910190F081BC
:10394000E02D6DE009957C01D801ED91FC9101908D
:10395000F081E02DC8016AE009959C012E0D3F1D04
:10396000C9011F910F91FF90EF900895CF93DF93BE
:10397000EC016115710519F420E030E00FC0DB01A6
:103980000D900020E9F71197A61BB70BE881F9818C
:103990000280F381E02DAD0109959C01C901DF9101
:1039A000CF9108954F925F927F928F929F92AF92A4
:1039B000BF92CF92DF92EF92FF920F931F93DF930C
:1039C000CF93CDB7DEB7A1970FB6F894DEBF0FBE89
:1039D000CDBF2C01742ECB01223008F42AE019A2AD
:1039E00031E2C32ED12CCC0EDD1E822E9924AA24C6
:1039F000BB24672D752FA50194010E94BC24790179
:103A00008A01C801B701A50194010E947624472DBF
:103A1000461B0894C108D1084A3014F4405D01C027
:103A2000495CF6014083E114F1040105110521F020
:103A30007E2C5F2DC801DDCFC201B6010E94B61CED
:103A4000A1960FB6F894DEBF0FBECDBFCF91DF9128
:103A50001F910F91FF90EF90DF90CF90BF90AF90AC
:103A60009F908F907F905F904F900895DC0121157B
:103A7000310541F4ED91FC910190F081E02D642F2E
:103A8000099508950E94D21C0895EF92FF920F931A
:103A90001F939A01E62EFF2400E010E0B801A70171
:103AA0000E94361D1F910F91FF90EF900895CF92C5
:103AB000DF92EF92FF920F931F93CF93DF93EC016E
:103AC0006A017B012115310541F4E881F9810190FA
:103AD000F081E02D642F09951FC02A303105D1F403
:103AE00077FF17C0E881F9810190F081E02D6DE248
:103AF00009958C0144275527BA014C195D096E09B7
:103B00007F09CE012AE00E94D21C9801280F391F9C
:103B100004C02AE00E94D21C9C01C901DF91CF9110
:103B20001F910F91FF90EF90DF90CF900895EF924B
:103B3000FF920F931F937B019A010027F7FC0095DA
:103B4000102FB801A7010E94571D1F910F91FF90E0
:103B5000EF900895CF92DF92EF92FF920F931F9311
:103B60006C017B019A010027F7FC0095102FB8012A
:103B7000A7010E94571D8C01C6010E94961C080FC8
:103B8000191FC8011F910F91FF90EF90DF90CF9008
:103B900008950E94B61C0895EF92FF920F931F9311
:103BA0007C010E94B61C8C01C7010E94961C080F64
:103BB000191FC8011F910F91FF90EF900895AF92C8
:103BC000BF92CF92DF92EF92FF920F931F93CF930A
:103BD000DF935C016B01EE24FF24C0E0D0E010C055
:103BE000D501ED91FC9100811181C601BE010E94B9
:103BF0007D20682FC501F8010995E80EF91E219670
:103C0000F60184819581C817D90750F3C701DF9168
:103C1000CF911F910F91FF90EF90DF90CF90BF90C9
:103C2000AF900895EF92FF920F931F937C010E9433
:103C3000DF1D8C01C7010E94961C9C01200F311FC3
:103C4000C9011F910F91FF90EF900895823000F508
:103C5000E82FF0E0EE0FFF1FED5BFA4F71836083FA
:103C6000882319F08130A1F408C0809169008C7F0D
:103C7000842B80936900E89A089580916900440F2D
:103C8000551F440F551F837F842B80936900E99A49
:103C90000895823080F4882319F0813021F402C025
:103CA000E89801C0E998E82FF0E0EE0FFF1FED5B08
:103CB000FA4F1182108208951F920F920FB60F9241
:103CC00011242F933F934F935F936F937F938F9321
:103CD0009F93AF93BF93EF93FF9380914305909190
:103CE0004405892B29F0E0914305F091440509959D
:103CF000FF91EF91BF91AF919F918F917F916F91C4
:103D00005F914F913F912F910F900FBE0F901F9099
:103D100018951F920F920FB60F9211242F933F9375
:103D20004F935F936F937F938F939F93AF93BF93C3
:103D3000EF93FF938091450590914605892B29F0DB
:103D4000E0914505F09146050995FF91EF91BF91EE
:103D5000AF919F918F917F916F915F914F913F9123
:103D60002F910F900FBE0F901F9018951F920F92DA
:103D70000FB60F9211242F933F938F939F93AF937E
:103D8000BF9380914B0590914C05A0914D05B0914A
:103D90004E0530914F050196A11DB11D232F2D5FBA
:103DA0002D3720F02D570196A11DB11D20934F05F1
:103DB00080934B0590934C05A0934D05B0934E0511
:103DC0008091470590914805A0914905B0914A0519
:103DD0000196A11DB11D8093470590934805A093BE
:103DE0004905B0934A05BF91AF919F918F913F9143
:103DF0002F910F900FBE0F901F9018958FB7F894CA
:103E000020914B0530914C0540914D0550914E0548
:103E10008FBFB901CA0108959FB7F8942091470553
:103E2000309148054091490550914A0586B5A89BB7
:103E300006C08F3F21F02F5F3F4F4F4F5F4F9FBF17
:103E4000542F432F322F2227280F311D411D511D82
:103E500082E0220F331F441F551F8A95D1F7B90105
:103E6000CA010895EF92FF920F931F93CF93DF93B0
:103E70007B018C010E940C1FEB010EC00E940C1FE5
:103E80006C1B7D0B685E7340C8F30894E108F10871
:103E900001091109C851DC4FE114F10401051105B4
:103EA00069F7DF91CF911F910F91FF90EF900895E7
:103EB000019739F0880F991F880F991F0297019772
:103EC000F1F70895789484B5826084BD84B58160EB
:103ED00084BD85B5826085BD85B5816085BDEEE612
:103EE000F0E0808181608083E1E8F0E010828081F1
:103EF00082608083808181608083E0E8F0E080815F
:103F000081608083E1EBF0E0808184608083E0EB7E
:103F1000F0E0808181608083EAE7F0E08081846066
:103F200080838081826080838081816080838081C2
:103F3000806880831092C1000895CF93DF93482F4B
:103F400050E0CA0189559F4FFC0134914D565F4F97
:103F5000FA018491882369F190E0880F991FFC0190
:103F6000EB58FF4FA591B491FC01E158FF4FC5916B
:103F7000D491662351F42FB7F8948C91932F909598
:103F800089238C93888189230BC0623061F42FB719
:103F9000F8948C91932F909589238C938881832B0F
:103FA00088832FBF06C09FB7F8948C91832B8C9386
:103FB0009FBFDF91CF910895833071F0843028F452
:103FC0008130A1F0823021F514C08630B1F0873005
:103FD000D1F08430E9F404C0809180008F7703C071
:103FE000809180008F7D80938000089584B58F77C5
:103FF00002C084B58F7D84BD08958091B0008F7715
:104000008093B00008958091B0008F7D8093B000C0
:104010000895FF920F931F93F62E482F50E0CA0188
:1040200085549F4FFC012491CA0189559F4FFC0183
:1040300014914D565F4FFA0104910023C9F02223D9
:1040400019F0822F0E94DC1FE02FF0E0EE0FFF1F1F
:10405000E158FF4FA591B4919FB7F894FF2021F448
:104060008C911095812302C08C91812B8C939FBFE2
:104070001F910F91FF9008950F931F93482F50E0C9
:10408000CA0185549F4FFC012491CA0189559F4F55
:10409000FC0104914D565F4FFA011491112319F45C
:1040A00020E030E015C0222319F0822F0E94DC1F8F
:1040B000812F90E0880F991F87579F4FFC01A59192
:1040C000B4918C9120E030E0802311F021E030E0C9
:1040D000C9011F910F910895FC0184819581681792
:1040E000790748F40190F081E02D309721F0E60F38
:1040F000F71F8081089580E00895FC0184819581F7
:104100006817790748F40190F081E02D309721F08D
:10411000E60FF71F8081089580E00895FC018081FB
:104120009181009729F420E030E040E050E004C0A5
:104130000E94A6029B01AC01B901CA010895CF9368
:10414000DF93FC01DB01848195814817590760F4F6
:10415000C081D1816D917C91CE01840F951F0E9409
:1041600015039C01009719F42FEF3FEF02C02C1BA1
:104170003D0BC901DF91CF910895CF93DF93FC01EF
:10418000848195814817590768F4C081D1817727C8
:1041900067FD7095CE01840F951F0E94F4029C016B
:1041A000009719F42FEF3FEF02C02C1B3D0BC90104
:1041B000DF91CF91089540E050E00E94BD20089526
:1041C0000F931F93CF93DF93FC018B014115510592
:1041D000F9F061157105E1F084819581281739079F
:1041E00018F0FB01108214C041505040EC01C21B7A
:1041F000D30B4C175D0708F4EA0160817181620FEF
:10420000731FC801AE010E940603C00FD11F1882A0
:10421000DF91CF911F910F9108950F931F93CF932B
:10422000DF93EC018B016F5F7F4F888199810E9442
:10423000B301009711F480E005C0998388831B8344
:104240000A8381E0DF91CF911F910F910895CF9361
:10425000DF93EC0188819981892B29F08A819B81E8
:104260008617970760F4CE010E940D21882341F044
:104270008C819D81892B19F4E881F981108281E07C
:10428000DF91CF910895EF92FF920F931F93CF93F9
:10429000DF93EC017B016C817D81E114F104C1F0BD
:1042A0004115510599F08A01060F171FB8010E94A8
:1042B0002721882369F0888199812C813D81820F93
:1042C000931FB7010E94FF021D830C8381E001C090
:1042D00080E0DF91CF911F910F91FF90EF900895B3
:1042E000EF92FF920F931F93DF93CF93CDB7DEB77B
:1042F00027970FB6F894DEBF0FBECDBF7C01CB0170
:104300008E010F5F1F4FB8014AE050E00E94610329
:10431000F80101900020E9F73197E01BF10BC7018C
:10432000B801AF010E94432127960FB6F894DEBF73
:104330000FBECDBFCF91DF911F910F91FF90EF90F6
:104340000895EF92FF920F931F93DF93CF9300D0C6
:1043500000D0CDB7DEB77C01862F90E08E010F5FD5
:104360001F4FB8014AE050E00E946103F80101903C
:104370000020E9F73197E01BF10BC701B801AF014D
:104380000E9443210F900F900F900F90CF91DF91DB
:104390001F910F91FF90EF900895DF93CF9300D07E
:1043A000CDB7DEB769831A82BE016F5F7F4F41E0F0
:1043B00050E00E9443210F900F90CF91DF9108951C
:1043C0006115710511F480E00895DB010D90002066
:1043D000E9F71197A61BB70BAD010E944321089581
:1043E000FB0160817181448155810E9443210895C0
:1043F000CF93DF93EC0188819981009711F00E949F
:104400005B01198218821D821C821B821A82DF9135
:10441000CF910895EF92FF920F931F93CF93DF9365
:10442000EC017B018A01BA010E942721882321F433
:10443000CE010E94F82107C01D830C8388819981D9
:10444000B7010E94FF02CE01DF91CF911F910F9122
:10445000FF90EF900895CF93DF93EC0119821882BB
:104460001B821A821D821C821E826115710551F009
:10447000DB010D900020E9F71197A61BB70BAD01EA
:104480000E940A22DF91CF9108950F931F93182F56
:10449000092F6115710559F0DB010D900020E9F736
:1044A0001197A61BB70BAD010E940A2202C00E9401
:1044B000F821812F902F1F910F910895EF92FF9275
:1044C0000F931F93DF93CF93CDB7DEB762970FB6ED
:1044D000F894DEBF0FBECDBF8C01CB01F801118275
:1044E0001082138212821582148216827E01089431
:1044F000E11CF11CB70150E00E946103C801B70143
:104500000E94452262960FB6F894DEBF0FBECDBF63
:10451000CF91DF911F910F91FF90EF900895EF924F
:10452000FF920F931F93DF93CF93CDB7DEB72997F9
:104530000FB6F894DEBF0FBECDBF8C01862FF801F9
:10454000118210821382128215821482168290E0E8
:104550007E010894E11CF11CB70150E00E949F030A
:10456000C801B7010E94452229960FB6F894DEBF14
:104570000FBECDBFCF91DF911F910F91FF90EF90B4
:104580000895BF92CF92DF92EF92FF920F931F9305
:10459000CF93DF93082FB92E6B017A01E90124171D
:1045A000350710F4EA017901802F9B2D6DE072E050
:1045B0000E942B22D60114968D919C9115978E15F1
:1045C0009F05D0F08C179D0708F4EC01D601ED9102
:1045D000FC911197EC0FFD1F108110826D917C9161
:1045E0006E0D7F1D802F9B2D0E944522D601ED91DF
:1045F000FC91EC0FFD1F1083802F9B2DDF91CF913D
:104600001F910F91FF90EF90DF90CF90BF90089592
:104610000F931F938C01FB01248135810E94C122DD
:10462000C8011F910F910895CF93DF93EC01FB0117
:104630008617970761F0608171816115710529F016
:10464000448155810E940A2202C00E94F821CE01B5
:10465000DF91CF910895FC01808191810E945B01DF
:104660000895BCD088F09F5790F0B92F9927B75183
:10467000A0F0D1F0660F771F881F991F1AF0BA9526
:10468000C9F712C0B13081F0C3D0B1E00895C0C005
:10469000672F782F8827B85F39F0B93FCCF386951C
:1046A00077956795B395D9F73EF490958095709579
:1046B00061957F4F8F4F9F4F0895E89409C097FBF6
:1046C0003EF490958095709561957F4F8F4F9F4FE9
:1046D0009923A9F0F92F96E9BB279395F69587952D
:1046E00077956795B795F111F8CFFAF4BB0F11F4F0
:1046F00060FF1BC06F5F7F4F8F4F9F4F16C0882397
:1047000011F096E911C0772321F09EE8872F762FCC
:1047100005C0662371F096E8862F70E060E02AF00D
:104720009A95660F771F881FDAF7880F96958795F9
:1047300097F90895990F0008550FAA0BE0E8FEEFCE
:1047400016161706E807F907C0F012161306E40755
:10475000F50798F0621B730B840B950B39F40A264E
:1047600061F0232B242B252B21F408950A2609F42C
:10477000A140A6958FEF811D811D089597F99F6730
:1047800080E870E060E008959FEF80EC08950024D9
:104790000A941616170618060906089500240A94A6
:1047A00012161306140605060895092E0394000C2C
:1047B00011F4882352F0BB0F40F4BF2B11F460FFBB
:1047C00004C06F5F7F4F8F4F9F4F089557FD9058E4
:1047D000440F551F59F05F3F71F04795880F97FBC5
:1047E000991F61F09F3F79F087950895121613067F
:1047F0001406551FF2CF4695F1DF08C016161706AE
:104800001806991FF1CF86957105610508940895E2
:10481000E894BB2766277727CB0197F908958ADFAD
:1048200008F48FEF08950BD0C0CFB1DF28F0B6DFCA
:1048300018F0952309F0A2CFA7CF1124EACFC6DF45
:10484000A0F3959FD1F3950F50E0551F629FF001A3
:10485000729FBB27F00DB11D639FAA27F00DB11DFC
:10486000AA1F649F6627B00DA11D661F829F222785
:10487000B00DA11D621F739FB00DA11D621F839F0C
:10488000A00D611D221F749F3327A00D611D231FE2
:10489000849F600D211D822F762F6A2F11249F5730
:1048A00050408AF0E1F088234AF0EE0FFF1FBB1F53
:1048B000661F771F881F91505040A9F79E3F5105F2
:1048C00070F05CCFA6CF5F3FECF3983EDCF38695AB
:1048D00077956795B795F795E7959F5FC1F7FE2B9D
:1048E000880F911D9695879597F90895629FD0013D
:1048F000739FF001829FE00DF11D649FE00DF11D9B
:10490000929FF00D839FF00D749FF00D659FF00D49
:104910009927729FB00DE11DF91F639FB00DE11D36
:10492000F91FBD01CF0111240895AA1BBB1B51E142
:1049300007C0AA1FBB1FA617B70710F0A61BB70B0F
:10494000881F991F5A95A9F780959095BC01CD01B4
:10495000089597FB092E07260AD077FD04D0E5DFDE
:1049600006D000201AF4709561957F4F0895F6F7F0
:10497000909581959F4F0895A1E21A2EAA1BBB1B0B
:10498000FD010DC0AA1FBB1FEE1FFF1FA217B3071B
:10499000E407F50720F0A21BB30BE40BF50B661F31
:1049A000771F881F991F1A9469F7609570958095F5
:1049B00090959B01AC01BD01CF010895EE0FFF1F43
:1049C0000590F491E02D09942F923F924F925F92BF
:1049D0006F927F928F929F92AF92BF92CF92DF920F
:1049E000EF92FF920F931F93CF93DF93CDB7DEB774
:1049F000CA1BDB0B0FB6F894DEBF0FBECDBF099408
:104A00002A88398848885F846E847D848C849B845E
:104A1000AA84B984C884DF80EE80FD800C811B816C
:104A2000AA81B981CE0FD11D0FB6F894DEBF0FBE9B
:104A3000CDBFED01089510E0C4EDD0E004C0FE014B
:104A40000E94E0242296C63DD107C9F7F894FFCF13
:104A50000041530025303258003030003000433DD3
:104A6000004C4C3D004C483D00534C3D0053483DEC
:104A7000004D53003D00443D0043503D0053503D28
:104A8000004F00636F7079004D430050004D55009A
:104A900053796E633A2000202D3E2053796E634691
:104AA0006163743A20002C20436C6F636B3A2000E2
:104AB0002C20546F6C3A20002C20506174744C658B
:104AC0006E3A200020002C2050756C73653A20004F
:104AD0002C20002C206D53746172743A20005369AD
:104AE000676E616C3A20002E2000205B005D005054
:104AF00061747465726E3A20002050003A20002ADA
:104B00005B00005550442046696C746572003B435D
:104B10003D003B53463D003B004954506172616D7E
:104B2000733A200020005620332E312E382053496E
:104B3000474E414C6475696E6F202D20636F6D7018
:104B4000696C6564206174204F63742032302032B8
:104B50003031352030303A34373A343300002000D9
:104B600054050000062C0100000000AC0F9B079CC0
:104B700007E41000000000AC0F9B079C075A0A00D6
:104B80000000000B079B079C079D0700000000002A
:104B900000020000000000881B411C1E1B4F1B2F41
:044BA0001B781B0063
:00000001FF
